:02000000312CA1
:0E000600213083120313FD00FD0B07280800B4
:08001400831603138514080094
:06001C00000000000800D6
:100022000F3083120313FC004730FD00FD0B17282D
:0A003200FC0B172800000000080076
:10003C00013083120313F100F11B2A28851C282898
:10004C00F1172928F10A2228F1137108F000080091
:0C005C0083160313851083128510080022
:0E0068008312031325088A0024088200080072
:1000760083120313F301FF30F5007508003A0319E4
:100086005828003085180130F4007409F000700813
:100096007305F1007108003A031954280130F20083
:1000A60059287408F300F5034028F2017208F0009D
:0200B600080040
:1000B80083120313D51B6228861363288617551BE2
:1000C8006728061368280617D51A6C2886126D2823
:1000D8008616551A712806127228061623187628CD
:1000E80006157728061186150E208611D5197E2843
:1000F80086137F2886175519832806138428061720
:10010800D518882886128928861655188D2806122B
:100118008E28061623189228061593280611861588
:100128000E208611231C9A2811209B2803200800E2
:1001380083120313D6010130D700D801D901013049
:10014800A7002708003A0319B7283B207008003A8F
:100158000319B628051CB4282708D6040130D70689
:10016800A70D2710A5283B207008003A0319C028BE
:10017800003005180130D8003B207008003A0319F8
:10018800C928003005180130D9002E205708580614
:10019800FF3003190030F1005908003AFF30031D01
:1001A8000030F0007008F1047108003A0319DD28E6
:0C01B800D601550884005608800008009D
:1001C40083120313D5010A201E207008003A031D70
:1001D400EE280130D5001529D601803056020318C7
:1001E40010290518F7287214F82872108518FC28AD
:1001F4000314FD280310721C0329031C0329721421
:1002040004297210721C09290130D50015295508DA
:10021400003A03190E291029D60AEF285508003A86
:0C022400031D15292E205508F0000800CD
:1002300083120313F5015508003A031D222975089E
:10024000F400C029A618262973102729731455080D
:10025000683CFF3003180030F100F0017318F00A19
:100260007008F1057E305502FF3003180030F000B1
:100270007008F1055508773AFF3003190030F00097
:100280007008F1057108003A03195A2969305502BE
:10029000F0000030F100D930F00705300318013EBE
:1002A000F1077008A4007108A50034208A110A1211
:1002B000F400C029D5035508F400A61E8F2955085F
:1002C000563EF00005300318013EF1007008A4000E
:1002D0007108A50034208A110A12F2007208F50094
:1002E000261974297310752973147208403CFF3065
:1002F00003180030F100F0017318F00A7008F105DE
:100300005B307202FF3003180030F0007008F10516
:100310007108003A03198E292030F507BE295508C7
:10032000D33EF00004300318013EF1007008A40031
:100330007108A50034208A110A12F2007208F50033
:100340002619A4297310A52973147208603CFF3084
:1003500003180030F100F0017318F00A7008F1057D
:100360007B307202FF3003180030F0007008F10596
:100370007108003A0319BE292030F5027508F4000F
:060380007408F000080003
:10038600831603178C1CC9290000C3298312031383
:100396004D0803178D0003134E0803178C008316B0
:1003A6008C130C150B08F0008B1355308D00AA30FA
:1003B6008D008C14F01BE1298B13E2298B170C118D
:0203C60008002D
:1003C8008312031323104D08D5005C202314080062
:1003D8008316031386110611061286120613861356
:1003E800831286110611861306138612061211202F
:1003F800112011208616061686150E20861111204A
:1004080086150E208611112086150E2086111120C2
:10041800061286150E208611112086150E208611CB
:100428008612861786150E20861111208613061649
:1004380086150E208611061286150E2086111120AB
:1004480086150E208611061686150E208611112097
:10045800061286150E2086118617061786160616AA
:0C04680086150E208611112023140800B8
:10047400013083120313D3000130D400D201A80148
:10048400E2207008003A031D492AD001FC2A5130A9
:10049400D5009C205108F03A031D5C2AD401E220C7
:1004A4007008003A031D582A0000512A5130D50023
:1004B4009C20902A5108E03A031D7A2AE220700811
:1004C400003A031D672A0000602A5130D5009C20A1
:1004D4005108F03A031D772AD401E2207008003A4B
:1004E40003196F2A5130D5009C200130A800902AAE
:1004F4005108773A031D8A2A0130D3005408003A80
:100504000319892AA618882AA614892AA610902ACB
:100514005108E13A031D902AE030D2002808003A3D
:100524000319A02A5108123A031D9A2ADF30D20077
:1005340051087C3A031DA02ADF30D2005108123A38
:10054400FF30031D0030F1005108593AFF30031DFC
:100554000030F0007108F0040319B92A0130D30007
:100564005408003A0319B82AA616B92AA612A618DE
:10057400BD2A7214BE2A72105108733AFF30031D4B
:100584000030F100F0017218F00A7108F005031947
:10059400CD2AD001FC2A5208003A031DD72AD301E0
:1005A4005108D50018217008D2005208E13A031D01
:1005B400E62A0130D3005408003A0319E62A261922
:1005C400E52A2615E62A26115208C83C0318EE2A05
:1005D4000130D300C830D2024D0884005208800094
:1005E4004E088400530880004F088400540880009B
:0A05F4000130D0005008F0000800AC
:0E05FE0083160313051485148312A60108004A
:10060C0083120313490803178D0083168C130C14E3
:0C061C0083120C08F1007108F0000800C7
:10062800323083120313CD003130CE003030CF008A
:100638003A2270080319AA2B3008003A0319AA2B8A
:100648004608333E840032088000C60A0319C70AE8
:1006580000304706031D322B11304606031D372B89
:100668001030C600C7013208123A031D4C2B023065
:100678004602F0000030031C013E4702F1007008FA
:10068800C6007108C7007008333E8400203080001F
:1006980080304706F00080307002031D552B013072
:1006A80046020318592BC601C70132080D3A031D2B
:1006B800AA2B0130C602031CC7034608333E840038
:1006C80020308000C60A0319C70A4508013A031DED
:1006D800702BC4011030AD004508023A031D782B79
:1006E8001230C4002230AD004408AC002C082D02A2
:1006F800031C982B2C08CD002B08333E84000008DF
:10070800CE00C32183120313AB0A1A30FC00F83061
:10071800FD00FD0B8D2BFC0B8D2B00002C082D06EE
:100728000319982BAC0A7A2B0230AF00AE012E08C1
:10073800333E8400203080002E08103A0319A62B7F
:0E074800AE0A9B2BC601C701C50AAB01080013
:100756000730831603139C009B0183129F010F3001
:1007660083169F00FC30860083128601FF308316B5
:10077600850083128501A901AA01AB010130C500DC
:100786000130AF00C601C7010130A0002030B30020
:10079600B4012030B3000030B400FF220230FB0069
:1007A6000430FC00BA30FD00FD0BD72BFC0BD72B19
:1007B600FB0BD72B0000EC210130D5005C200C3060
:1007C600D5005C200E30D5005C20AE012E08333EED
:1007D6008400203080002E08103A0319F42BAE0A4C
:0407E600E92B0800F3
:1007EA00831203134908013A031DFE2B8030C90006
:1007FA00152C4908023A031D052CC030C900152CD6
:10080A004908033A031D0C2C9430C900152C4908D9
:10081A00043A031D132CD430C900152C8030C900AA
:10082A004A03F0004908F0077008C9007008D500AB
:10083A005C202310CC014C084B0784000008003AC6
:10084A0003192F2C4C084B0784000008CD00E42123
:08085A00CC0A202C2314080035
:10086200AB230330A100210845020318532C051EB7
:10087200502C14232F08C9000130CA003330CB009A
:10088200F5230230FB000430FC00BA30FD00FD0B02
:10089200482CFC0B482CFB0B482C0000522C03303C
:1008A200C500342C0130D5005C20A10A2108450284
:1008B2000318D22C051D7F2CA2012208333EC8004A
:1008C2002208C90006230313480884007008800028
:1008D2001A30FC00F830FD00FD0B6D2CFC0B6D2C6A
:1008E20000002208103A0319782CA20A5E2C01306B
:1008F200C9000130CA003330CB00F5238519C42C5E
:100902001230A2002908333EC8002208C90006237B
:1009120003134808840070088000A90A0319AA0A70
:100922001A30FC00F830FD00FD0B952CFC0B952CC9
:1009320000002208223A0319A02CA20A832CA90142
:10094200AA010130C9000130CA003330CB00F523BF
:1009520086140530FB000F30FC00F130FD00FD0B6A
:10096200B02CFC0BB02CFB0BB02C86100530FB001E
:100972000F30FC00F130FD00FD0BBD2CFC0BBD2C3B
:10098200FB0BBD2C7F2C0230FB000430FC00BA3084
:10099200FD00FD0BCA2CFC0BCA2CFB0BCA2C000061
:0409A200572CD22CD0
:1009A600D1340034CD34CB34C934CA34D434D334FE
:1009B600D234D034CE34CC34EB346034003400340A
:1009C600DE34DD340034DC34713431340034003448
:1009D60000347A347334613477343234DB3400349F
:1009E600633478346434653434343334DB3400347B
:1009F600203476346634743472343534003400343A
:100A06006E346234683467347934363400340034F2
:100A160000346D346A347534373438340034003475
:100A26002C346B3469346F34303439340034003448
:100A36002E342F346C343B3470342D34003400346F
:100A46000034273400345B343D3400340034E13460
:100A5600DD34D5345D3400345C3400340034003485
:100A660000340034003400340034D8340034003408
:100A7600E2340034E634E334003400340034D9344C
:100A8600DA34E9343534E734E834EA34E534D33457
:100A96002B34D7342D342A34D634E434003400349D
:060AA60000340034CF34DF
:100AAC00D1340034CD34CB34C934CA34D4340034CA
:100ABC00D234D034CE34CC34EB347E3400340034E5
:100ACC00DE34DD340034DC34513421340034003471
:100ADC0000345A345334413457344034DB3400340A
:100AEC00433458344434453424342334DB34003414
:100AFC0020345634463454345234253400340034C3
:100B0C004E3442344834473459345E340034003463
:100B1C0000344D344A34553426342A3400340034ED
:100B2C003C344B3449344F342934283400340034A9
:100B3C003E343F344C343A3450345F340034003457
:100B4C000034223400347B342B3400340034E13450
:100B5C00DD34D5347D3400347C340034003400343E
:100B6C0000340034003400340034D8340034003401
:100B7C00E2340034E634E334003400340034D93445
:100B8C00DA34E9343534E734E834EA34E534D33450
:100B9C002B34D7342D342A34D634E4340034003496
:060BAC0000340034CF34D8
:100BB20031340034343437340034003400343034C7
:100BC2002E34323435343634383400340034003480
:0A0BD2002B3433342D342A34393427
:04400E00623F03000A
:00000001FF
